S01A000064656D6F70726F675F73746D3332663734362E737265638E
S315080080000805002075A10008BDA10008C1A1000847
S31508008010C5A10008C9A10008CDA1000800000000FC
S31508008020000000000000000000000000D1A10008C8
S31508008030D5A1000800000000D9A100089B9A0008F5
S31508008040DDA10008E1A10008E5A10008E9A10008F2
S31508008050EDA10008F1A10008F5A10008F9A10008A2
S31508008060FDA1000801A2000805A2000809A200084F
S315080080700DA2000811A2000815A2000819A20008FE
S315080080801DA2000821A2000825A2000829A20008AE
S315080080902DA2000831A2000835A2000839A200085E
S315080080A03DA2000841A2000845A2000849A200080E
S315080080B04DA2000851A2000855A2000859A20008BE
S315080080C05DA2000861A2000865A2000869A200086E
S315080080D06DA2000871A2000875A2000879A200081E
S315080080E07DA2000881A2000885A2000889A20008CE
S315080080F08DA2000891A2000895A2000899A200087E
S315080081009DA20008A1A20008A5A20008A9A200082D
S31508008110ADA20008B1A20008B5A20008B9A20008DD
S31508008120BDA20008C1A20008C5A20008C9A200088D
S31508008130CDA20008D1A20008D5A20008D9A200083D
S31508008140DDA20008E1A20008E5A20008E9A20008ED
S31508008150EDA20008F1A20008F5A20008F9A200089D
S31508008160FDA2000801A3000805A3000809A300084A
S315080081700DA3000811A3000815A3000800000000BD
S3150800818019A300081DA3000821A3000825A30008B9
S3150800819029A300082DA3000831A3000835A3000869
S315080081A039A300083DA3000841A3000845A3000819
S315080081B049A300084DA3000851A3000855A30008C9
S315080081C059A300085DA30008EE11AA5510B50400CE
S315080081D0002C01D1012035E0A0690028FFD1606F8D
S315080081E0002805D1002084F87000200000F06AFB02
S315080081F024206067206800684008400021680860FD
S31508008200200000F0B1F8012801D101201AE0606AC7
S31508008210002802D0200000F06FFA2068406830F489
S315080082209040216848602068806830F02A002168FC
S3150800823088602068006850F0010021680860200006
S3150800824000F0C7FA10BD2DE9F84306000D0014002A
S315080082501F00B06F202840F08480002D03D0200036
S3150800826080B2002801D101207CE096F87000012830
S3150800827001D1022076E0012086F870000020F06720
S315080082802220B06700F03CFB8046A6F85840A6F8C6
S315080082905A40B068B0F5805F0BD13069002804D128
S315080082A040F2FF10A6F85C0023E0FF20A6F85C0069
S315080082B01FE0B06800280AD13069002803D1FF20E2
S315080082C0A6F85C0015E07F20A6F85C0011E0B0680F
S315080082D0B0F1805F0AD13069002803D17F20A6F863
S315080082E05C0006E03F20A6F85C0002E00020A6F845
S315080082F05C00B6F85C90B068B0F5805F04D1306970
S31508008300002801D1002401E02C000025002086F871
S31508008310700013E03068406A19EA00002070641C97
S3150800832007E0002CF6D13068406A19EA0000288078
S31508008330AD1CB6F85A00401EA6F85A00B6F85A0000
S3150800834000280AD00097434600222021300000F07A
S3150800835061FA0028E5D0032004E02020B067002059
S3150800836000E00220BDE8F28338B5040000210025AC
S31508008370A2682069024360690243E06902432068F3
S315080083800368DFF8440303401A4320680260206844
S31508008390426832F44052E068024320684260A269AB
S315080083A0206A02432068806830F4306002432068FF
S315080083B082602068DFF81423904216D1DFF8100394
S315080083C0006810F00300002805D0022805D006D35F
S315080083D0032806D007E00120D3E00220D1E00420DC
S315080083E0CFE00820CDE01020CBE02068DFF8E422BB
S315080083F0904217D1DFF8D802006810F00C00002868
S3150800840006D0042808D0082804D00C2806D007E08F
S315080084100020B6E00220B4E00420B2E00820B0E074
S315080084201020AEE02068AC4A904216D1A8480068F1
S3150800843010F03000002806D0102808D0202804D0D4
S31508008440302806D007E000209BE0022099E00420AF
S3150800845097E0082095E0102093E020689F4A904214
S3150800846016D19B48006810F0C000002806D04028A6
S3150800847008D0802804D0C02806D007E0002080E075
S3150800848002207EE004207CE008207AE0102078E0D4
S315080084902068934A904219D18D48006810F44070BC
S315080084A0002809D0B0F5807F0AD0B0F5007F05D046
S315080084B0B0F5407F06D007E0002062E0022060E0C9
S315080084C004205EE008205CE010205AE02068854A17
S315080084D0904219D17E48006810F44060002809D0FF
S315080084E0B0F5806F0AD0B0F5006F05D0B0F5406FD3
S315080084F006D007E0012044E0022042E0042040E0E4
S3150800850008203EE010203CE02068774A904219D1C6
S315080085106F48006810F44050002809D0B0F5805F15
S315080085200AD0B0F5005F05D0B0F5405F06D007E089
S31508008530002026E0022024E0042022E0082020E093
S3150800854010201EE02068694A904219D160480068E8
S3150800855010F44040002809D0B0F5804F0AD0B0F595
S31508008560004F05D0B0F5404F06D007E0002008E0E0
S31508008570022006E0042004E0082002E0102000E0C3
S315080085801020E269B2F5004F4FD1C0B2002808D0DA
S31508008590012811D002281AD0042821D008282AD068
S315080085A032E000F097FC6168490811EB4001606809
S315080085B0B1FBF0F189B228E000F097FC6168490840
S315080085C011EB40016068B1FBF0F189B21DE060680B
S315080085D0474911EB50016068B1FBF0F189B214E02C
S315080085E000F03DFC6168490811EB40016068B1FB89
S315080085F0F0F189B209E06068400810F580306168DA
S31508008600B0FBF1F189B200E001254FF6F072B1F145
S315080086101000904207D20A40C1F34200024392B2C8
S315080086202068C26048E0012546E0C0B2002808D0AC
S31508008630012810D0022818D004281FD0082827D0CF
S315080086402FE000F047FC616810EB51006168B0FB51
S31508008650F1F189B226E000F048FC616810EB5100A0
S315080086606168B0FBF1F189B21CE06068214911EB41
S3150800867050016068B1FBF0F189B213E000F0EFFB3E
S31508008680616810EB51006168B0FBF1F189B209E04D
S315080086906068400810F500406168B0FBF1F189B2E6
S315080086A000E00125B1F110004FF6F072904202D2B7
S315080086B02068C16000E00125002020660020606671
S315080086C02800C0B232BD0000F369FFEF0010014078
S315080086D0903802400044004000480040004C0040EA
S315080086E0005000400014014000780040007C004023
S315080086F00048E8010024F40090F82410C90707D5BB
S3150800870001684A6832F40032816A0A4301684A609D
S3150800871090F82410890707D501684A6832F4803230
S31508008720C16A0A4301684A6090F82410490707D5C8
S3150800873001684A6832F48022016B0A4301684A607C
S3150800874090F82410090707D501684A6832F40042F0
S31508008750416B0A4301684A6090F82410C90607D598
S3150800876001688A6832F48052816B0A4301688A601C
S3150800877090F82410890607D501688A6832F40052F1
S31508008780C16B0A4301688A6090F82410490613D51C
S3150800879001684A6832F48012016C0A4301684A602B
S315080087A0016CB1F5801F07D101684A6832F4C0022E
S315080087B0416C0A4301684A6090F82410090607D5F7
S315080087C001684A6832F40022816C0A4300684260F4
S315080087D070471CB504000020E06700F091F803001C
S315080087E02068006800070CD57FF07E4000900022C4
S315080087F05FF40011200000F00DF8002801D00320D6
S3150800880007E0202060672020A067002084F8700019
S31508008810002016BD2DE9F04105000E0090461F0008
S31508008820069C2868C0693040B04201D1012000E0AA
S3150800883000204146C9B2884241D114F1010FF0D057
S3150800884000F05EF8C01B844201D3002C14D12868BE
S31508008850006830F4D0702968086028688068400885
S31508008860400029688860202068672020A8670020C3
S3150800887085F87000032023E0286800684007D0D5F3
S315080088802868C0690005CCD54FF4006029680862DD
S315080088902868006830F4D0702968086028688068FD
S315080088A04008400029688860202068672020A8675B
S315080088B02020E867002085F87000032000E00020EB
S315080088C0BDE8F081704730B4002513E050F8042B5A
S315080088D0D30744BFA9F101039A18091F042942F8CE
S315080088E0045BFAD213468C0744BF15809B1CC90744
S315080088F048BF1D7050F8041B0029E7D130BC7047EB
S3150800890001480068704700BF000100202DE9FC41BE
S3150800891004000025002C01D10120F6E12078C007CB
S315080089206DD5DFF8E005016811F00C01042909D0BE
S31508008930006810F00C0008280ED1DFF8CC05006896
S31508008940400209D5DFF8B8050068800357D5606886
S31508008950002854D10120D8E16068B0F5803F06D1DF
S31508008960DFF89C05016851F48031016026E06068F3
S3150800897000280AD1DFF88805016831F480310160E2
S31508008980016831F48021016018E06068B0F5A02F15
S315080089900AD1DFF86C05016851F48021016001688D
S315080089A051F48031016009E0DFF85405016831F4BB
S315080089B080310160016831F4802101606068002817
S315080089C00ED0FFF79DFF0600DFF834050068800328
S315080089D015D4FFF795FF801B6528F5D3032094E18E
S315080089E0FFF78EFF0600DFF818050068800306D536
S315080089F0FFF786FF801B6528F5D3032085E12078DD
S31508008A00800720D5DFF8FC04016811F00C0F09D0A7
S31508008A10006810F00C0008282ED1DFF8EC04006876
S31508008A20400229D4DFF8D8040168890704D5E1682B
S31508008A30012901D0012068E1016831F0F8012269B5
S31508008A4051EAC20101602078000759D560690028FB
S31508008A5043D0DFF8B874386850F001003860FFF783
S31508008A604FFF0600386880074AD4FFF749FF801B86
S31508008A700328F7D3032048E1E06800281AD0DFF876
S31508008A808064306850F001003060FFF739FF070056
S31508008A903068800706D4FFF733FFC01B0328F7D3D7
S31508008AA0032032E1306830F0F800216950EAC1004D
S31508008AB03060C8E7DFF84874386840084000386016
S31508008AC0FFF71EFF060038688007BCD5FFF718FFBA
S31508008AD0801B0328F7D3032017E1DFF830743868C2
S31508008AE0400840003860FFF70BFF0600386880072B
S31508008AF006D5FFF705FF801B0328F7D3032004E1FB
S31508008B002078400740F18280DFF810643068C000A2
S31508008B1009D4306850F080503060306810F08050CA
S31508008B20009000980125DFF8F8733868C00511D45D
S31508008B30386850F480703860FFF7E2FE804638687F
S31508008B40C00507D4FFF7DCFEB0EB08006528F6D3AE
S31508008B500320DAE0A068012806D1DFF8C803016817
S31508008B6051F00101016025E0A06800280AD1DFF86C
S31508008B70B4030168490849000160016831F004013D
S31508008B80016017E0A06805280AD1DFF89803016894
S31508008B9051F004010160016851F00101016009E02A
S31508008BA0DFF880030168490849000160016831F06F
S31508008BB004010160A068002810D0FFF7A1FE070095
S31508008BC0DFF860030068800719D4FFF799FEC01B19
S31508008BD041F289318842F3D3032096E0FFF790FEED
S31508008BE00700DFF840030068800708D5FFF788FE0E
S31508008BF0C01B41F289318842F3D3032085E0EDB2E8
S31508008C00012D03D1306830F080503060A06900280B
S31508008C107AD0DFF8F002006810F00C0008284CD073
S31508008C20A069022836D1DFF8D852286830F080705B
S31508008C302860FFF765FE06002868800106D5FFF75D
S31508008C405FFE801B0328F7D303205EE0E169206AF4
S31508008C500143606A51EA8011A06A4008401E51EA41
S31508008C600041E06A51EA006151F00051DFF89802CC
S31508008C700160286850F080702860FFF741FE040004
S31508008C802868800140D4FFF73BFE001B0328F7D372
S31508008C9003203AE0DFF86852286830F080702860D0
S31508008CA0FFF72EFE0400286880012DD5FFF728FE61
S31508008CB0001B0328F7D3032027E0DFF84C020068DF
S31508008CC0A16901291ED010F48001E269914219D1E7
S31508008CD010F03F01226A914214D147F6C071014053
S31508008CE0626AB1EB821F0DD110F44031A26A5208B4
S31508008CF0521EB1EB024F05D110F07060E16AB0EB7D
S31508008D00016F01D0012000E00020BDE8F6812DE9C1
S31508008D10F04104000D000020002C01D101209CE048
S31508008D20DFF80462306810F00F00A8420BD23068F2
S31508008D300009000128433060306810F00F00A8428F
S31508008D4001D0012089E02078800719D520784007CE
S31508008D5005D5DFF8B001016851F4E05101602078CB
S31508008D60000705D5DFF89C01016851F460410160F0
S31508008D70DFF890110A6832F0F002A06802430A6030
S31508008D802078C00733D56068012806D1DFF870015E
S31508008D900068800310D401205FE06068022805D1CE
S31508008DA057480068800107D4012056E054480068F7
S31508008DB0800701D4012050E0524F3968890889009C
S31508008DC0606801433960FFF79BFD8046386810F0FC
S31508008DD00C006168B0EB810F09D0FFF791FDB0EB8D
S31508008DE0080041F289318842F0D3032035E0306823
S31508008DF010F00F0085420BD23068000900012843A5
S31508008E003060306810F00F00A84201D0012024E03D
S31508008E102078400706D53B490A6832F4E052E068F4
S31508008E2002430A602078000707D53648016831F4FE
S31508008E306041226951EAC201016000F010F83B491D
S31508008E40304A1268C2F30312895CC8403149086087
S31508008E503148006800F070F80020BDE8F08110B5D0
S31508008E6000200020002000202648006810F00C0092
S31508008E70002804D0042804D0082804D025E0244873
S31508008E8024E02B4822E0204C226812F03F0220689A
S31508008E90400209D52068C0F388102549A1FB0001C6
S31508008EA0002300F06FF808E02068C0F3881018491E
S31508008EB0A1FB0001002300F065F82168C1F3014118
S31508008EC0491C4900B0FBF1F000E0114810BD1148FB
S31508008ED00068704780B5FFF7FAFF1649094A126815
S31508008EE0C2F38222895CC84002BD80B5FFF7EFFF56
S31508008EF01049044A1268C2F34232895CC84002BD6E
S31508008F0000380240083802400438024074380240EB
S31508008F100024F4000400002000000020403802402D
S31508008F200070004070380240003C02408CA10008E6
S31508008F3000127A00B4A1000810B504004FF47A7044
S31508008F400D490978B0FBF1F00C490968B1FBF0F05E
S31508008F5000F09EF9002801D001200CE0102C09D25F
S31508008F60002221005FF0FF3000F081F90448046018
S31508008F70002000E0012010BD0800002004000020A9
S31508008F8000000020BBBBE1B1B2F5803F80F07E80D7
S31508008F90022A1ED98C46B1FBF2F102FB11C31B044F
S31508008FA043EA1043B3FBF2FC02FB1C3380B240EAEF
S31508008FB00343B3FBF2F002FB103240EA0C400023F5
S31508008FC07047022A05D98446B0FBF2F002FB10C2AC
S31508008FD070474AB105D100F0010249085FEA30003E
S31508008FE0704700220023704700F090B90B0002007A
S31508008FF0002100207047904271EB030CF6D3B3F5BD
S31508009000803F2FD2F0B5B3FA83F7B1FA81F4A7F10E
S315080090100F0E3D1B5340CEF1200602FA0EF2F34125
S315080090205340B5F10F0746D80F3C2C444140C4F1D4
S315080090302006A040F1414140B1FBF3F603FB1611AF
S31508009040A2FB0645001BA94102D2761E801859418B
S3150800905080EA010221FA0EF362FA0EF200215A4062
S315080090603046F0BD30B4B1FBF3FC03FB1C11A2FB88
S315080090700C45001BA94103D2ACF1010C80185941DB
S3150800908030BC02460B46604600217047B2F1807F2D
S3150800909065D3F0B5B2FA82F7B1FA81F4C7F10F06D3
S315080090A03D1B22FA06F307F1110EF24120355A400C
S315080090B0B5F10F07B8D94140C4F12006A040F141E7
S315080090C04140B1FBF3FC03FB1C11A2FB0C45001B42
S315080090D0A94103D2BCF1010C801859410F2F12D3B4
S315080090E00F3FC90341EA5041B1FBF3F603FB1611E2
S315080090F0A2FB0645D4EBC030A94102D2761E8018E1
S31508009100594146EACC3C07B34140C7F12006B8406E
S31508009110F1414140B1FBF3F603FB1611A2FB0645EC
S31508009120001BA94102D2761E8018594180EA010225
S3150800913021FA0EF3C7F1200462FA0EF20CFA07F0D0
S315080091405A402CFA04F13043F0BD80EA010221FAB4
S315080091500EF3002162FA0EF260465A40F0BD8C46C4
S31508009160B1FBF2F102FB11C31B0243EA1063B3FB26
S31508009170F2FC02FB1C331B024CEA002043EA106394
S31508009180B3FBF2FC02FB1C331B024CEA002043EA49
S315080091901063B3FBF2FC02FB1C331B024CEA0020F3
S315080091A043EA1063B3FBF2FC02FB1C324CEA0020D4
S315080091B00023704710F007003F4B1A684FF6FF016F
S315080091C00A403E4951EA00210A431A6070473A4864
S315080091D00068C0F302207047020052B2002A04D485
S315080091E00901374A40B2115407E00901354A40B22D
S315080091F010F00F00104400F8041C704710B410F06B
S315080092000700D0F10703052B01D3042301E0D0F1B1
S315080092100703041D072C01D2002000E0C01E01240C
S3150800922014FA03F35B1E1940814014FA00F0401E3D
S315080092301040084310BC704780B5411EB1F1807FCD
S3150800924001D301200EE0401E1F4908600F215FF080
S31508009250FF30FFF7C1FF00201C49086007201C49A2
S315080092600860002002BD80B5FFF7A4FF01BD70B5F8
S3150800927004000D0016000020FFF7A9FF32002900A0
S31508009280FFF7BCFF0100200040B2FFF7A5FF70BD45
S3150800929080B5FFF7D1FF02BD042805D10C48016847
S315080092A051F00401016004E00948016831F0040145
S315080092B001607047000000000CED00E00000FA05B0
S315080092C000E400E018ED00E014E000E018E000E03B
S315080092D010E000E080B500F001F801BD704730B439
S315080092E00EE00268436802440830DC0744BFA9F16F
S315080092F00104E31852F8045B43F8045B091FF9D12B
S3150800930050F8041B0029ECD130BC704770470000A8
S3150800931038B50400002C01D10120AEE094F82000F5
S31508009320002802D1200000F015FA2068006830F005
S31508009330020021680860FFF7E3FA05002068406824
S3150800934080070DD5FFF7DCFA401B0B28F6D3606AB9
S3150800935050F400306062052084F8200001208CE07B
S315080093602068006850F0010021680860FFF7C8FA15
S31508009370050020684068C0070DD4FFF7C1FA401BF6
S315080093800B28F6D3606A50F400306062052084F832
S315080093902000012071E0207E012806D1206800689F
S315080093A050F080002168086005E02068006830F009
S315080093B0800021680860607E012806D12068006860
S315080093C050F040002168086005E02068006830F029
S315080093D0400021680860A07E012806D12068006840
S315080093E050F020002168086005E02068006830F029
S315080093F0200021680860E07E012806D12068006800
S3150800940030F010002168086005E02068006850F018
S31508009410100021680860207F012806D120680068AE
S3150800942050F008002168086005E02068006830F000
S31508009430080021680860607F012806D12068006856
S3150800944050F004002168086005E02068006830F0E4
S31508009450040021680860A168E068014320690143A7
S31508009460606901436068401E01432068C1610020AD
S315080094706062012084F82000002032BD30B4026802
S3150800948090F820201300DBB2012B03D0D2B2022AB7
S3150800949040F07F80594AD2F8000250F00100C2F825
S315080094A00002D2F8000230F47C50C2F80002D2F86A
S315080094B000024B6A50EA0320C2F8000201200B7D25
S315080094C013F01F0310FA03F3D2F81C029843C2F8EC
S315080094D01C02C869002816D1D2F80C029843C2F8B3
S315080094E00C02486902EBC000CC684D68C5EA044422
S315080094F0C0F84042486902EBC0008C680D68C5EAAE
S315080095000444C0F84442C869012816D1D2F80C02AE
S315080095101843C2F80C02486902EBC0000C684D6893
S31508009520C5EA0444C0F84042486902EBC0008C68AA
S31508009530CD68C5EA0444C0F844428869002805D1C4
S31508009540D2F804029843C2F8040204E0D2F80402EE
S315080095501843C2F804020869002805D1D2F8140293
S315080095609843C2F8140204E0D2F814021843C2F869
S315080095701402086A012804D1D2F81C020343C2F86F
S315080095801C32D2F8000240084000C2F8000200204F
S3150800959004E0416A51F480214162012030BC7047E1
S315080095A038B5040094F82000012821D1022084F857
S315080095B02000206800684008400021680860FFF71E
S315080095C09FF9050020684068C0070DD5FFF798F990
S315080095D0401B0B28F6D3606A50F400306062052001
S315080095E084F82000012008E000206062002004E0E2
S315080095F0606A50F400206062012032BD00640040B9
S3150800960030B490F820402500EDB2012D03D0E4B225
S31508009610022C40F0988000290AD10468E46814F006
S31508009620030F10D1416A51F40011416201208FE005
S315080096300468246914F0030F05D1416A51F4001136
S315080096404162012084E004680D012C44D4F8B0413D
S3150800965014F0040494609468002C07D104680D0182
S315080096602C44D4F8B041640D146006E004680D017A
S315080096702C44D4F8B041E408546004680D012C4425
S31508009680D4F8B04114F00204D46004680D012C44E7
S31508009690D4F8B44114F00F04146104680D012C4485
S315080096A0D4F8B441C4F30724946104680D012C442A
S315080096B0D4F8B441240C546102680C012244D2F84F
S315080096C0B8211A7002680C012244D2F8B821120A8D
S315080096D05A7002680C012244D2F8B821120C9A700A
S315080096E002680C012244D2F8B821120EDA70026818
S315080096F00C012244D2F8BC211A7102680C012244DA
S31508009700D2F8BC21120A5A7102680C012244D2F816
S31508009710BC21120C9A7102680C012244D2F8BC21B1
S31508009720120EDA71002906D10168C96851F02001C4
S315080097300068C16005E00168096951F02001006808
S315080097400161002004E0416A51F480214162012050
S3150800975030BC704770470000BFF34F8FB6490A68A0
S3150800976012F4E062B54802430A60BFF34F8F00BFA8
S31508009770FDE780B500F00DF800F0CDF801BD80B525
S3150800978000F021F800F02AF901BD80B5FFF7E4FFE3
S3150800979001BD80B5AA48AB4901604FF461414160FB
S315080097A0002181600021C160002101610C21416115
S315080097B0002181610021C16100210162002141620D
S315080097C0FEF704FD01BD70B59F4C2078002815D121
S315080097D09E4D280000F037F8012833D12878002854
S315080097E030D0287841282DDA00F053F998490860D6
S315080097F00120207000209749087023E0954D934E6C
S3150800980028783044401C00F01EF8012811D1287829
S31508009810401C287028783178884213D1002020709F
S315080098207078FF280ED1287802280BD1FFF7ADFFF4
S3150800983008E000F02EF9864909686431814201D2B0
S315080098400020207070BD80B50100002301227C48ED
S31508009850FEF7F9FCC0B2002801D1012000E0002083
S3150800986002BDF8B504000D0016001F00FFF732FB15
S315080098704FF47A71B0FBF1F1002200E0521C10009F
S31508009880C0B2122845D2744B200080B294465FFAC3
S315080098908CFC13F81CC096465FFA8EFE03EB4E0E40
S315080098A09EF801E01EEB0C0C1CF1010C0CFB00F001
S315080098B0B1FBF0FC00FB1C100028DFD1200080B2B1
S315080098C094465FFA8CFC13F81CC096465FFA8EFE27
S315080098D003EB4E0E9EF801E01EEB0C0C1CF1010C7E
S315080098E00CFB00F0B1FBF0F0288028880028C5D0D2
S315080098F0288840F2014C6045C0DA1000C0B213F85F
S3150800990010003070D2B203EB420040783870012064
S3150800991000E00020F2BD30B58BB00020ADF80200A3
S3150800992000208DF8010000208DF8000040F26765E0
S315080099306B460DF101020DF102014FF4FA70FFF7C3
S3150800994090FF464C4648206000202076002060762E
S315080099500020A0760120E07600202077002060779E
S315080099600020A0600020E0609DF80100401E000471
S3150800997020619DF80000401E00056061BDF80200E8
S3150800998060602000FFF7C4FC002D02D46D05354841
S3150800999005E025F00045ED0055F0040532480021A4
S315080099A0069100210791012108912900090C0191CE
S315080099B0ADB202950100090C039180B20490002013
S315080099C00590012009900E200A9001A92000FFF7B2
S315080099D055FD2000FFF7E4FD0BB030BD30B589B06A
S315080099E040F2676400256B4602AA00211B48FFF770
S315080099F007FE00281ED1002C07D40298A0420DD1DC
S31508009A00049800280AD1012508E024F000440398A8
S31508009A10A04203D10498042800D10125EDB2012DF6
S31508009A2008D19DF80000FF2804D10698022801D124
S31508009A30FFF7ABFE09B030BD0CED00E00400FA05F7
S31508009A400C00002000480040050100208C00002082
S31508009A50F800002004010020A4A00008D00000207F
S31508009A60006400400400E0FFFCFF1F0080B5FFF71C
S31508009A702EFA4FF47A71B0FBF1F0FFF709FC0420D7
S31508009A80FFF70AFC002200215FF0FF30FFF7EFFB2B
S31508009A9001BD80B5FEF734FF02BD80B500F004F8BD
S31508009AA0FFF718FC01BD000003480168034A127855
S31508009AB089180160704700BF0001002008000020D7
S31508009AC0F8B40022002200220022002337E00A27E9
S31508009AD004E0DFF8E4219042F9D10927FFB213F038
S31508009AE00302D2B2920097403E431A00920845F804
S31508009AF02260DFF8C8512A68A2434E68F60300D5EB
S31508009B0022432A60DFF8B8512A68A2434E68B60392
S31508009B1000D522432A60DFF8AC512A68A2434E6872
S31508009B20F60200D522432A60DFF89C512A68A24330
S31508009B304E68B60201D5144322002A605B1C102B1E
S31508009B4080F0AD80012515FA03F20C6814409442A2
S31508009B50F4D14A68012A08D04A68022A05D04A6818
S31508009B60112A02D04A68122A16D1866803271A00D3
S31508009B70D2B252009740BE43CF681A00D2B2520002
S31508009B8097403E43866042689D40AA434D68C5F3A8
S31508009B9000159D402A434260C66803251A00D2B2C2
S31508009BA0520015FA02F296438F681A00D2B2520092
S31508009BB097403E43C6604A68022A02D04A68122A7B
S31508009BC017D11A00D20800EB8202166A0F2713F083
S31508009BD00702D2B292009740BE430F6913F00702FC
S31508009BE0D2B2920097403E431A00D20800EB820296
S31508009BF0166206681A00D2B252009540AE430D7935
S31508009C0015F003051A00D2B2520095402E4306609D
S31508009C104A68D20092D52D4A156855F480451560D4
S31508009C20126812F480420092009A294D1A0092088E
S31508009C3055F822600F2713F00302D2B2920097401C
S31508009C40BE43244A904201D1002747E7224A904260
S31508009C5001D1012742E7214A904201D102273DE777
S31508009C601F4A904201D1032738E71E4A904201D184
S31508009C70042733E71C4A904201D105272EE71B4AE1
S31508009C80904201D1062729E7194A904201D10727B0
S31508009C9024E7184A90427FF41CAF08271EE7F1BC58
S31508009CA07047D2B2002A02D089B2816102E089B235
S31508009CB0090481617047000000240240003C01400D
S31508009CC0043C0140083C01400C3C01404438024039
S31508009CD00838014000000240000402400008024023
S31508009CE0000C024000100240001402400018024016
S31508009CF0001C02400020024080B500F007F8FFF77C
S31508009D0038FD00F010F9FFF73AFDFAE780B500F0E4
S31508009D1009F800F02DF900F009F8FFF7A7FE00F0A2
S31508009D20FBF801BD744875490860704780B592B064
S31508009D303022002106A800F026F91422002101A8E5
S31508009D4000F021F96E48016851F080510160006801
S31508009D5010F08050009000986A48016851F440411C
S31508009D600160006810F440400090009801200690B9
S31508009D705FF4A020079002200C905FF480000D90FD
S31508009D8008200E904FF4D8700F90022010900220F1
S31508009D90119006A8FEF7BAFD002800D0FEE700F0ED
S31508009DA0FDF8002800D0FEE70F200190022002905F
S31508009DB0002003904FF4A05004904FF48050059073
S31508009DC0072101A8FEF7A3FF002800D0FEE713B07D
S31508009DD000BD38B586B04A48016851F08051016027
S31508009DE0016811F080510591059947490A6852F4AE
S31508009DF080420A60096811F4804105910599434932
S31508009E000A6852F002020A600A6812F00202059213
S31508009E10059A0A6852F008020A60096811F00801F2
S31508009E2005910599016851F480210160016811F4D2
S31508009E30802105910599016851F00071016000685B
S31508009E4010F00070059005980320FFF70CFA002221
S31508009E5000217FF00B00FFF70AFA002200217FF0AD
S31508009E600A00FFF704FA002200217FF00900FFF735
S31508009E70FEF9002200217FF00400FFF7F8F900221E
S31508009E8000217FF00300FFF7F2F9002200217FF09E
S31508009E900100FFF7ECF9002200215FF0FF30FFF721
S31508009EA0E6F9802000900120019000200290002011
S31508009EB00390174C69462000FFF702FE4FF44075E1
S31508009EC000950220019000200290032003900720AD
S31508009ED0049069460F48FFF7F3FD009502200190AC
S31508009EE00020029003200390092004906946200070
S31508009EF0FFF7E6FD07B030BD0080000808ED00E07A
S31508009F004038024000700040443802403038024071
S31508009F1000040240000C024080B50022802111484E
S31508009F20FFF7BFFE01BD38B5FFF7B3FD04000E4DC0
S31508009F302868201AB0F5FA7F13D30C490878002848
S31508009F4007D101200870012280210648FFF7A9FEE3
S31508009F5006E000200870002280210248FFF7A1FED3
S31508009F602C6031BD00040240FC00002006010020E0
S31508009F7080B50320FFF777F90020FEF7DDFFFFF72E
S31508009F8028FF002002BD10B5044610460A460146C1
S31508009F90204600F03FF8204610BD00007CB50020A2
S31508009FA01B48016851F080510160006810F080502C
S31508009FB000900098154E306850F480303060FEF7F7
S31508009FC09FFC0500104C2068C00308D4FEF798FCD7
S31508009FD0401B40F2E9318842F4D3032013E030688D
S31508009FE050F400303060FEF78BFC050020688003D3
S31508009FF008D4FEF785FC401B40F2E9318842F5D3C8
S3150800A000032000E0002076BD047000400070004088
S3150800A0104038024062F30F2262F31F42401810F0E4
S3150800A020030308D0C91A1FD3DB0748BF00F8012D60
S3150800A03028BF20F8022D130030B4144615461039EF
S3150800A04028BF20E93C00FAD8490728BF20E90C00B8
S3150800A05048BF40F8042D890028BF20F8022D48BFC4
S3150800A06000F8012D30BC7047C91818BF00F8012D3B
S3150800A070CB0728BF00F8012D7047000010B5074927
S3150800A08079441831064C7C44163404E00A68081DE5
S3150800A090114488470146A142F8D110BD500000007E
S3150800A0A070000000050206020603070308030903F9
S3150800A0B009040A040B040C040C050D050E050F050E
S3150800A0C00F061006100710084EF68851CEF200014A
S3150800A0D0086840F470000860BFF34F8FBFF36F8FB6
S3150800A0E04FF00070E1EE100A70470000DBE7FFFF53
S3150800A0F0FC0000000C00002000000000E3F1FFFF58
S3150800A1000C000000A4000000000000200000000071
S3150800A11000F00DF8002801D0FFF7B0FFAFF300807C
S3150800A1200020AFF30080FFF7E7FD00F002F80120FA
S3150800A130704700F001B800000746384600F002F8FC
S3150800A140FBE7000080B5AFF30080024A1100182033
S3150800A150ABBEFBE7260002000448016851F4700113
S3150800A16001605FF0006002490860704788ED00E012
S3150800A17008ED00E002488546024880470248004745
S3150800A1800805002059A100089DA10008000000004C
S3150800A190000000000102030406070809AFF3008067
S3150800A1A0FFF792FFFFF7B4FF100000000024F40049
S3150800A1B0010000000000000001020304FFF7FEBFD3
S3150800A1C0FFF7FEBFFFF7FEBFFFF7FEBFFFF7FEBFB5
S3150800A1D0FFF7FEBFFFF7FEBFFFF7FEBFFFF7FEBFA5
S3150800A1E0FFF7FEBFFFF7FEBFFFF7FEBFFFF7FEBF95
S3150800A1F0FFF7FEBFFFF7FEBFFFF7FEBFFFF7FEBF85
S3150800A200FFF7FEBFFFF7FEBFFFF7FEBFFFF7FEBF74
S3150800A210FFF7FEBFFFF7FEBFFFF7FEBFFFF7FEBF64
S3150800A220FFF7FEBFFFF7FEBFFFF7FEBFFFF7FEBF54
S3150800A230FFF7FEBFFFF7FEBFFFF7FEBFFFF7FEBF44
S3150800A240FFF7FEBFFFF7FEBFFFF7FEBFFFF7FEBF34
S3150800A250FFF7FEBFFFF7FEBFFFF7FEBFFFF7FEBF24
S3150800A260FFF7FEBFFFF7FEBFFFF7FEBFFFF7FEBF14
S3150800A270FFF7FEBFFFF7FEBFFFF7FEBFFFF7FEBF04
S3150800A280FFF7FEBFFFF7FEBFFFF7FEBFFFF7FEBFF4
S3150800A290FFF7FEBFFFF7FEBFFFF7FEBFFFF7FEBFE4
S3150800A2A0FFF7FEBFFFF7FEBFFFF7FEBFFFF7FEBFD4
S3150800A2B0FFF7FEBFFFF7FEBFFFF7FEBFFFF7FEBFC4
S3150800A2C0FFF7FEBFFFF7FEBFFFF7FEBFFFF7FEBFB4
S3150800A2D0FFF7FEBFFFF7FEBFFFF7FEBFFFF7FEBFA4
S3150800A2E0FFF7FEBFFFF7FEBFFFF7FEBFFFF7FEBF94
S3150800A2F0FFF7FEBFFFF7FEBFFFF7FEBFFFF7FEBF84
S3150800A300FFF7FEBFFFF7FEBFFFF7FEBFFFF7FEBF73
S3150800A310FFF7FEBFFFF7FEBFFFF7FEBFFFF7FEBF63
S3150800A320FFF7FEBFFFF7FEBFFFF7FEBFFFF7FEBF53
S3150800A330FFF7FEBFFFF7FEBFFFF7FEBFFFF7FEBF43
S3150800A340FFF7FEBFFFF7FEBFFFF7FEBFFFF7FEBF33
S3150800A350FFF7FEBFFFF7FEBFFFF7FEBFFFF7FEBF23
S7050800A19DB4
